:10000000C228B4006220200821040319BD28B720AB
:1000100084133408800664000D280E28A00A0319F2
:10002000A10F0B288006BD283708A0003508A100C5
:100030000130A200A30164003C20031C2F28A20B66
:100040001B28FF30A30703181B28A007031CA107C8
:10005000031CBD28C830A2000030A3001B28472085
:100060000830A30048203C20A20C3628A30B3228DD
:100070004820031422080800360884003408841736
:1000800080048413000533193406FF3E080033173B
:10009000330D0639A0005620A100A00A5620331FB8
:1000A0008A283313A00002309C208A2800308A005E
:1000B00020088207013496340334363400345D342A
:1000C0000C34FA34FF3A84178005BD2803178D00DD
:1000D00083168C130C1483120C08BD2803178C0094
:1000E00083168C130C1555308D00AA308D008C149E
:1000F0008C1878280C11BD28A301A200FF30A2079C
:10010000031CA307031CBD280330A100E6308A208E
:100110007E28A101FB3EA000A109FF30031C93280B
:10012000A00703189028A0076400A10F90280000E2
:1001300008000310A10CA00CFF3E0318992820080A
:10014000BD281030A800A101A001A70CA60C031C1B
:10015000AF282208A00723080318230FA107A10C2A
:10016000A00CA50CA40CA80BA5282408BD28A00948
:10017000A109A00A0319A10A08008313031383121B
:1001800064000800831607309F00053083128A013F
:100190006620BA0006308A016620BB0007308A015B
:1001A0006620BC0008308A016620BD0009308A0143
:1001B0006620BE00BF0164008A11861CE128013060
:1001C000C00064008A118618E7280430C000861336
:1001D0003A08A600A7010430A200A3018A01A120C9
:1001E000B8002508B9003808A0003908A100063079
:1001F000840080308A01012006133B08A600A70175
:100200000430A200A3018A01A120B8002508B9008A
:100210003808A0003908A1000630840040308A0167
:10022000012086123C08A600A7010430A200A30109
:100230008A01A120B8002508B9003808A0003908B3
:10024000A1000630840020308A01012006123D08FA
:10025000A600A7010430A200A3018A01A120B800D2
:100260002508B9003808A0003908A100063084002C
:1002700010308A01012086113E08A600A701043033
:10028000A200A3018A01A120B8002508B9003808FE
:10029000A0003908A1000630840008308A0101203E
:1002A0000A308A017C2064008A11061D682A6400D5
:1002B0008A11871D1D2A64008A11071D302A6400D7
:1002C0008A11871CF72964008A11071C0A2A640016
:1002D0008A11851ED12964008A11051EE429640053
:1002E0008A11851DAB2964008A11051DBE29640091
:1002F0008A11851C852964008A11051C98296400CF
:100300008A11071F432A8A01E728BF0A64003F08B1
:1003100040028A11031D8E29BA0ABF016400FF3012
:100320003A028A11031C9629FE30BA008A01E72896
:10033000BF0A64003F0840028A11031DA129BA03C5
:10034000BF0164004B303A028A110318A9294B30CF
:10035000BA008A01E728BF0A64003F0840028A11F8
:10036000031DB429BB0ABF016400FF303B028A11A0
:10037000031CBC29FE30BB008A01E728BF0A6400C9
:100380003F0840028A11031DC729BB03BF01640057
:100390004B303B028A110318CF294B30BB008A0136
:1003A000E728BF0A64003F0840028A11031DDA29CA
:1003B000BC0ABF016400FF303C028A11031CE22921
:1003C000FE30BC008A01E728BF0A64003F084002F3
:1003D0008A11031DED29BC03BF0164004B303C02B0
:1003E0008A110318F5294B30BC008A01E728BF0A9F
:1003F00064003F0840028A11031D002ABD0ABF01A4
:100400006400FF303D028A11031C082AFE30BD0043
:100410008A01E728BF0A64003F0840028A11031DD1
:10042000132ABD03BF0164004B303D028A1103183B
:100430001B2A4B30BD008A01E728BF0A64003F0831
:1004400040028A11031D262ABE0ABF016400FF3044
:100450003E028A11031C2E2AFE30BE008A01E728C4
:10046000BF0A64003F0840028A11031D392ABE03F7
:10047000BF0164004B303E028A110318412A4B3001
:10048000BE008A01E728031705308D0003133A08E0
:100490008A016E20031706308D0003133B088A0182
:1004A0006E20031707308D0003133C088A016E206D
:1004B000031708308D0003133D088A016E200317CF
:1004C00009308D0003133E088A016E208A01E72857
:1004D0000630B6000130B4000630B3001430B70067
:1004E000B5018A0114208A11031C982A073C8A113D
:1004F000031D712A8A0114208A11031C982ABE0048
:100500008A0114208A11031C982ABD008A01142034
:100510008A11031C982ABC008A0114208A11031C2A
:10052000982ABB008A0114208A11031C982ABA0059
:040530008A01E7282D
:02400E00753FFC
:0A420A0096009600960096009600BC
:00000001FF
